:1004000000010102020203030404040505060606B6
:1004100007070808080909090A0A0B0B0B0C0C0D41
:100420000D0D0E0E0F0F0F101011111112121213CD
:100430001314141415151616161717181818191959
:10044000191A1A1B1B1B1C1C1D1D1D1E1E1F1F1FE6
:100450002020202121222222232324242425252672
:10046000262627272728282929292A2A2B2B2B2CFF
:100470002C2C2D2D2E2E2E2F2F303030313131328D
:10048000323333333434353535363636373738381A
:100490003839393A3A3A3B3B3B3C3C3D3D3D3E3EA8
:1004A0003E3F3F4040404141414242434343444438
:1004B00045454546464647474848484949494A4AC6
:1004C0004B4B4B4C4C4C4D4D4E4E4E4F4F4F505056
:1004D00050515152525253535354545555555656E8
:1004E0005657575858585959595A5A5A5B5B5C5C79
:1004F0005C5D5D5D5E5E5E5F5F606060616161620C
:10050000626263636464646565656666666767679F
:1005100068686969696A6A6A6B6B6B6C6C6C6D6D33
:100520006E6E6E6F6F6F70707071717172727273C8
:10053000737474747575757676767777777878785E
:100540007979797A7A7A7B7B7B7C7C7C7D7D7E7EF7
:100550007E7F7F7F8080808181818282828383838E
:100560008484848585858686868787878888888928
:1005700089898A8A8A8B8B8B8C8C8C8D8D8D8E8EC3
:100580008E8E8F8F8F909090919191929292939363
:1005900093949494959595969696979797979898FF
:1005A000989999999A9A9A9B9B9B9C9C9C9C9D9D9F
:1005B0009D9E9E9E9F9F9FA0A0A0A0A1A1A1A2A240
:1005C000A2A3A3A3A3A4A4A4A5A5A5A6A6A6A6A7E3
:1005D000A7A7A8A8A8A9A9A9A9AAAAAAABABABAB87
:1005E000ACACACADADADADAEAEAEAFAFAFAFB0B02D
:1005F000B0B1B1B1B1B2B2B2B3B3B3B3B4B4B4B5D4
:10060000B5B5B5B6B6B6B6B7B7B7B8B8B8B8B9B97C
:10061000B9B9BABABABBBBBBBBBCBCBCBCBDBDBD27
:10062000BDBEBEBEBEBFBFBFC0C0C0C0C1C1C1C1D4
:10063000C2C2C2C2C3C3C3C3C4C4C4C4C5C5C5C582
:10064000C6C6C6C6C7C7C7C7C8C8C8C8C9C9C9C932
:10065000CACACACACACBCBCBCBCCCCCCCCCDCDCDE5
:10066000CDCECECECECECFCFCFCFD0D0D0D0D1D199
:10067000D1D1D1D2D2D2D2D3D3D3D3D3D4D4D4D450
:10068000D5D5D5D5D5D6D6D6D6D6D7D7D7D7D8D807
:10069000D8D8D8D9D9D9D9D9DADADADADADBDBDBC2
:1006A000DBDBDCDCDCDCDCDDDDDDDDDDDEDEDEDE7F
:1006B000DEDFDFDFDFDFE0E0E0E0E0E0E1E1E1E13D
:1006C000E1E2E2E2E2E2E2E3E3E3E3E3E4E4E4E4FE
:1006D000E4E4E5E5E5E5E5E5E6E6E6E6E6E7E7E7C1
:1006E000E7E7E7E8E8E8E8E8E8E9E9E9E9E9E9E986
:1006F000EAEAEAEAEAEAEBEBEBEBEBEBEBECECEC4D
:10070000ECECECEDEDEDEDEDEDEDEEEEEEEEEEEE16
:10071000EEEFEFEFEFEFEFEFF0F0F0F0F0F0F0F0E2
:10072000F1F1F1F1F1F1F1F2F2F2F2F2F2F2F2F3AF
:10073000F3F3F3F3F3F3F3F3F4F4F4F4F4F4F4F481
:10074000F5F5F5F5F5F5F5F5F5F6F6F6F6F6F6F652
:10075000F6F6F6F7F7F7F7F7F7F7F7F7F7F8F8F829
:10076000F8F8F8F8F8F8F8F9F9F9F9F9F9F9F9F900
:10077000F9F9F9FAFAFAFAFAFAFAFAFAFAFAFAFBDB
:10078000FBFBFBFBFBFBFBFBFBFBFBFBFBFCFCFCB6
:10079000FCFCFCFCFCFCFCFCFCFCFCFCFDFDFDFD95
:1007A000FDFDFDFDFDFDFDFDFDFDFDFDFDFDFDFE78
:1007B000FEFEFEFEFEFEFEFEFEFEFEFEFEFEFEFE59
:1007C000FEFEFEFEFEFEFEFFFFFFFFFFFFFFFFFF40
:1007D000FFFFFFFFFFFFFFFFFFFFFFFFFFFFFFFF29
:1007E000FFFFFFFFFFFFFFFFFFFFFFFFFFFFFFFF19
:1007F000FFFFFFFFFFFFFFFFFFFFFFFFFFFFFFFF09
:020000001CC022
:100008001FB6260C371C481C591CE42DF52D52FC34
:10001800E09552FCF095F370F460C89553FC05C068
:100028000094969808BA1FBE189508BA969A1FBEEB
:1000380018954FED4DBF40E048BB4FEF47BB4CE331
:1000480042BB43E441BB332793E040E04093710057
:10005800CC2440E04FBD4BBF40E448BF49BF49E016
:100068004EBD40E04BBD47E24ABD45E043BF65E8B1
:100078005AEF48EC4A95F1F75A95D9F76A95C1F7BE
:1000880041E74093720047EC409373004CEB409378
:1000980074004AE04093750040EA042F46E8142FA4
:1000A80041E0242FF6D0CFD0316078947ED15091A2
:1000B8007100541731F04093710043E0A42E326070
:1000C80019C0542FAA20B1F431FF03C040E5B42E63
:1000D80004C0BB2079F444E1B42E513009F420D097
:1000E800523009F428D0543009F431D0583009F48A
:1000F80035D03D7F48B741FF0BC0427048BF4EE93D
:1001080042BFA395AA2009F0AA94BB2009F0BA948B
:1001180032FF04C0CC2011F43B7F316002D1C6CF3E
:1001280032FD01C022C027D036D054D073D00EF48F
:100138008AD0AFD01AC032FD01C017C01CD00EF053
:1001480036D048D067D00EF47ED0A3D00EC032FD92
:1001580001C00BC0973049F0939507C032FD01C02C
:1001680004C0913011F09A9500C03460316044E1C8
:10017800C42EAA270895692FE8946A9559F0D0E00B
:10018800CAE6C61BD04048814423B9F344274883B4
:100198006894F3CF089568E0691B15D043954A30F9
:1001A80021F4442748836A95C1F74883089568E095
:1001B800691B09D04A954F3F21F449E048836A9565
:1001C800C1F7488308954427D0E0C2E6C60FD41F7C
:1001D80048810895D0E0C3E609911127222766E0F7
:1001E800499103D06A95E1F70895D02EE12EF22EB9
:1001F800000F111F221F0AD009D008D00D0D1E1D97
:100208002F1D040F40E0141F241F0895DD0CEE1C61
:10021800FF1C0895E89440E404174BE414074CE4E9
:10022800240728F000E41BE42CE468940BC044E69F
:10023800041740E0140740E0240720F404E610E027
:1002480020E0689408955F93D02EE12EF22E6AE0A4
:10025800D0E0C0E6442749936A95E9F768E1DD0CE8
:10026800EE1CFF1C87E0D0E0CAE64A915FB75F93B7
:100278004D5F43FF48815F915FBF441F889444FDF1
:1002880008944F7048838A9581F76A9541F75F9182
:1002980008955F93D0E0CAE667E0442749936A95DA
:1002A800E9F768E1422F469540936C00412F479546
:1002B80040936B00402F479540936A00B0F4D0E01C
:1002C800CDE6488150917200450F4993488150917D
:1002D8007300451F4993488150917400451F499305
:1002E800488150917500451F4993D0E0C1E777E0F8
:1002F8004A91479548837A95D9F76A95F9F6D0E0F7
:10030800CCE660E84991460F6627F8946990661E26
:100318007990761E8990861E9990961E78945F91A2
:10032800089532FF0FC0503069F4A5FF07C033FDB0
:1003380023C03860CC2049F0CA9407C033FF1CC0E2
:10034800377F03C0377F30FF17C06AE0D0E0C0E6D0
:10035800E894499132FF07C0691729F4689433FF7C
:1003680002C0442705C0442311F416F44AE06894F7
:1003780004D06A9571F73E7F08956F9364E04295C3
:10038800441F10F0909801C0909A919A85E08A9540
:10039800F1F791988AE08A95F1F76A9589F789E1EA
:1003A8008A95F1F790986F9108954427859B41604D
:0E03B800839B4260849B4460829B4860089552
:00000001FF
